:06000000008077022CD005
:03000B0002247557
:0300130002234A7B
:03001B000225714A
:03002300022C7636
:10002B003202534D50544520496E746572666163BC
:10003B0065202020286329203139393520202041A3
:10004B006C636F726E204D63427269646520496EFA
:10005B00632E2020200D534D50544520496E74655E
:10006B00726661636520432056352E30300D00C219
:10007B00AF75D00075816C43B0FF4390FF7589213C
:10008B00758804758DFD758BFDD28E7589237598DA
:10009B00D0787FE4F6D8FD751800751E149000001B
:1000AB007400F0A3A883B820F974FF90E800F090D7
:1000BB001523F090E000F0901522F075A015781E36
:1000CB0090E000E0F20890E800E0F2D294D296754E
:1000DB0066057401904002F0D297901522E044100F
:1000EB00F090E000F01201E5902E4212026D902E7E
:1000FB005512026D121C221221A61221539080025E
:10010B0074B5F0122DD9C294122DE7D294740090CD
:10011B004002F0122DE7C294122DE7D294122DE774
:10012B007401904002F0C294122DE7D294122DE785
:10013B00C294122DE7D294122DD9122DD9122DD98A
:10014B00122DD9122DD9122DD9122DD9122DD9121A
:10015B002DD9122DD9122DD9902E6812026D75B88A
:10016B000075A811D2AF751200901522E054FBF068
:10017B0090E000F012159812160FC215C23FD20173
:10018B00302A04C201C22C75816C300144C28CC26E
:10019B0092758A00754C00C204D246D28CD2A990BB
:1001AB002E4212026D902E6812026D1205473023FB
:1001BB0003120C7D30011212030A3004EEC204B29A
:1001CB00941207A230010280E2C28CC2A9C246D2AD
:1001DB009220220302172302196DD2387A301202B1
:1001EB000B7A3012020B7A3812020B7A8012020B46
:1001FB007A0612020B7A0C12020B7A0112020B22F4
:10020B00C0F030381775F00075A0A07802E230E727
:10021B000700D5F0F30202277800EAF2D0F022C0F3
:10022B00F030381A75F00075A0A07802E230E707BD
:10023B0000D5F0F302024975A0A07801EAF2D0F0E4
:10024B0022C0F030381975F00075A0A07802E230AA
:10025B00E70700D5F0F302026A75A0A07803E2D09D
:10026B00F022740093A312028BFA740093A32AFA60
:10027B0012020B740093A36006FA12022A80F42276
:10028B0083227FBF93D37A8512020BE55175F00061
:10029B00600475F00A842430FA12022AE5F0243047
:1002AB00FA12022A7A3A12022AE55275F000600419
:1002BB0075F00A842430FA12022AE5F02430FA127F
:1002CB00022A7A3A12022AE55375F000600475F09F
:1002DB000A842430FA12022AE5F02430FA12022A98
:1002EB007A2E12022AE55475F000600475F00A8428
:1002FB002430FA12022AE5F02430FA12022A2230B4
:10030B003A08E56930E00312032E303B08E569300B
:10031B00E103120465303C08E56930E2031204681E
:10032B00C23A22E562C39561F4B412005003020491
:10033B0064A86275A01C74FEF2F5F075A01B740125
:10034B00F20875A01CE56BF225F0F5F075A01BE427
:10035B00F20875A01C7428F225F0F5F075A01BE4CB
:10036B00F20875A01CE56AF225F0F5F075A01BE408
:10037B00F20875A01CE551F225F0F5F075A01BE411
:10038B00F20875A01CE5F0C313F275A01B7401F203
:10039B000875A01C74FEF2F5F075A01B7401F20831
:1003AB0075A01CE56BF225F0F5F075A01BE4F208C7
:1003BB0075A01C7428F225F0F5F075A01BE4F2086B
:1003CB0075A01CE56A2401F225F0F5F075A01BE47D
:1003DB00F20875A01CE552F225F0F5F075A01BE4B0
:1003EB00F20875A01CE5F0C313F275A01B7401F2A3
:1003FB000875A01C74FEF2F5F075A01B7401F208D1
:10040B0075A01CE56BF225F0F5F075A01BE4F20866
:10041B0075A01C7428F225F0F5F075A01BE4F2080A
:10042B0075A01CE56A2402F225F0F5F075A01BE41B
:10043B00F20875A01CE553F225F0F5F075A01BE44E
:10044B00F20875A01CE5F0C313F275A01B7401F242
:10045B000888629060057406F022C23B22E562C3F5
:10046B009561F4B40C005003020546A86275A01CFC
:10047B0074FEF2F5F075A01B7401F20875A01CE573
:10048B006BF225F0F5F075A01BE4F20875A01C7457
:10049B0028F225F0F5F075A01BE4F20875A01CE519
:1004AB006A2404F225F0F5F075A01BE4F20875A0A0
:1004BB001C901563E0F225F0F5F075A01BE4F20833
:1004CB0075A01CE5F0C313F275A01B7401F208753F
:1004DB00A01C74FEF2F5F075A01B7401F20875A058
:1004EB001CE56BF225F0F5F075A01BE4F20875A086
:1004FB001C7428F225F0F5F075A01BE4F20875A02A
:10050B001CE56A2405F225F0F5F075A01BE4F20852
:10051B0075A01C901564E0F225F0F5F075A01BE4B6
:10052B00F20875A01CE5F0C313F275A01B7401F261
:10053B000888629060057406F0C23C22E559655A42
:10054B00600812057A20232680F2302D0512288BA5
:10055B00800EE563656460081206A020231080F20C
:10056B00E55F656060081206CB80F585605F2275DC
:10057B00A01EA959E3FA75A01DE3FB0559C239C2A8
:10058B0029BB0006EA20280F803CEA30E73690159D
:10059B005CF0D22802069FC228B4FE0DF51CF51D97
:1005AB00751800751E1402069FB480005005751D4A
:1005BB0000805E751DFDD22490155DC0E0E4F0D087
:1005CB00E002065CD229AD1DBDFE030205E8BD00AD
:1005DB0003020638BDFD0302065C02069FBB000248
:1005EB00801AF5F090155CE0251CC313B5F005D20D
:1005FB002302069F74551216F802069F851EA0A8AB
:10060B0018F2251CF51C088818B80002051E0206F6
:10061B009F90155CE075831C856282F07401758375
:10062B001BF00582E5616582602485826220391E9C
:10063B0075831C856282EAF0EB75831BF00582E5FE
:10064B0061658260098582629060057406F002061E
:10065B009F30290990155DE0C313FAC22990155DEF
:10066B00E02AF0758318855E82EAF0302406C224F6
:10067B00740180027400758317F00582E55D658255
:10068B00600F85825E90800274B5F09080057406D1
:10069B00F002069F2275A01AA963E3FA75A019E36D
:1006AB00FB056375831F855C82EAF00582E55B655C
:1006BB0082600385825C202002D299D23902058A9E
:1006CB0075A016A85FE2055FB4FE0BD230C231C233
:1006DB0032C2330207A130300AB41302D231C23016
:1006EB000207A1303110B42000505F901563F0C2A7
:1006FB0031D2320207A130320B901564F0C232D2E4
:10070B00330207A130334BF87A11901563E02AFAC4
:10071B00901564E02A547FC398702F901564E0F80D
:10072B00901563E09015652582F58274003583F58D
:10073B0083E8F0D23C30E504D234800375671E9019
:10074B001522E054FDF090E000F0C231C232C2330A
:10075B008044C231C232C233F5F0B4FF0B2020FD0E
:10076B007598D8752C00D22C302C12052C7405B52D
:10077B002C0B2020FD7598D8752C00D22CE5F0752C
:10078B00831F855C82F00582E55B65826003858251
:10079B005C202002D2992230033120901875660517
:1007AB007401904002F0D297901522E04410F09023
:1007BB00E000F08016D566137400904002F0C297EB
:1007CB00901522E054EFF090E000F020930F2037CB
:1007DB0019D23774BF75F00A1216AB800D30370A79
:1007EB00C23774BF75F00B1216AB75A015791FE3EA
:1007FB00FB90E800E0F36B5B60357B0833502EC059
:10080B00E090E000E030E61C75F00030E70375F097
:10081B001020E50343F04074B12BFAEBF9121F01E2
:10082B00D0E0800974B12BFA121F89D0E0DBCD75B3
:10083B00A015781EE2FA90E000E0F26A5AFAEA5448
:10084B001F606330E029D291C201201510200019DE
:10085B00C23F302214301F11121B55800C103F0267
:10086B008007C2AF121B55D2AFC200C21580373002
:10087B00E109202B06D200C291802B30E308C2AFD6
:10088B00D215D2AF802030221530E406C2AFD2157C
:10089B00D2AF30E211D201D291121FD5800830E2D3
:1008AB0005D201121FD5227851E6084608460846A4
:1008BB0060121208D07002800B12095D60067D1663
:1008CB00DDFE80F522900000E06026F975650030B2
:1008DB00257D20267A7E107F008E828F83E0B4FFE9
:1008EB0002806CF5F07851E6B5F00280104060D9CB
:1008FB0002805C74082EFEEF3400FF80DCA3E0B4B2
:10090B00FF02804BF5F008E6B5F002800440408012
:10091B00DEA3E0B4FF028037F5F008E6B5F0028005
:10092B0004402C80CAA3E0B4FF028023F5F008E654
:10093B00B5F0028004401880B6E565B4000DA3AB9A
:10094B0082AC83901520EBF0A3ECF0056580A0E55D
:10095B006522901520E0FBA3E0FCE565B4000302E3
:10096B0009A78B828C83E0FEA3E0FFA3E0F9700361
:10097B00020996A3E0B4FF030209AAB48000500356
:10098B000209D9020A34D565028011EB2408FB90C9
:10099B001520F0A3EC3400FCF002096DE56522E5AF
:1009AB005CC3955BF489F0B5F00050030209A78E88
:1009BB00828F83A85C75A01FE0F2A308D9FA885C2C
:1009CB00202002D299D565030209A7020996E56298
:1009DB00C39561F489F0B5F00050030209A78E822C
:1009EB008F83A86275A01CE0D2E7F275A01B74017F
:1009FB00F2D903088022A308D902800FE075A01C4E
:100A0B00F275A01B7400F2A308D9F1E075A01CF2DB
:100A1B0075A01B7401F2A30888629060057406F040
:100A2B00D565030209A7020996E55EC3955DF489B6
:100A3B00F0B5F00050030209A78E828F83A85EE009
:100A4B0075A018F275A0177401F2A308D903020957
:100A5B0096E075A018F275A0177400F2A308D9F1EF
:100A6B00885E90800274B5F09080057406F0D565B1
:100A7B00030209A7020996E538C4540FF5F0E539CE
:100A8B0054F045F030E72530E622543FF5F0B43F03
:100A9B00028024900007E0B5F002801B901500E067
:100AAB00600AFAA3E0B5F002800DDAF790153EE488
:100ABB00F0A3F0A3F08008901536E5F0F0D21622E3
:100ACB00901536E0F5F0A3E53AC4540FF9E53B5425
:100ADB003049F025F0F5F0A3E53CC4540FF9E53DA2
:100AEB00543049F025F0543FF5F0901536E5F0F011
:100AFB0022901536E0F5F0E53EC4540FF9E53F546E
:100B0B003049B5F002800B90153EE4F0A3F0A3F052
:100B1B008020C21E7903783E75A015E2F5F0E0B592
:100B2B00F0028002D21EF2121E7ED9EF301E03029B
:100B3B001E86227400B5520DB5530AB551077403C6
:100B4B00B55400500122901526E060F9FA7400F0BC
:100B5B00A3A85E12214CB4030040F875A018E0D294
:100B6B00E7F2FB75A0177401F20875A0187408F270
:100B7B002BFB75A0177400F20875A018EBF275A08B
:100B8B00177400F208885E75A080790274B5F3754E
:100B9B00A08079057406F3A3DAB9C21B229000007A
:100BAB00E07005D226020C0175F000900005E0C341
:100BBB0095F0900003F075F008900006E095F0902A
:100BCB000004F0900000E0C226C39402500280267D
:100BDB0004FA750513750400850406850507790766
:100BEB00120C73EAFB120C047907120C73DBF67907
:100BFB0005120C73DAE2D22522C082C083A80585C8
:100C0B0004A0850782850683E0F5F0E2C395F0C06A
:100C1B00D0120C4BE0F5F0E2D0D095F0C0D0120C16
:100C2B004BE0F5F0E2D0D095F0C0D0120C4BE0F5D4
:100C3B00F0E2D0D095F04003120C5FD083D082222B
:100C4B00C0E01582E582B4FF02158318B8FF0215C8
:100C5B00A0D0E0227908E2F5F0E0F2E5F0F0A3088D
:100C6B00B8000205A0D9EF22E72408F719E73400F2
:100C7B00F722901400E0B44203020EC5543F232325
:100C8B00900C8F73020D9700020FB00002105100F1
:100C9B000210620002107F00020D8F000210900004
:100CAB000210B6000210F00002118100021369005D
:100CBB0002138D000213B3000213CD000213D900EF
:100CCB0002142C0002148B00021564000215400064
:100CDB0002151A000214F100021112000211320067
:100CEB000212EC0002140C0002141B000213580039
:100CFB00020D8F00020D8F00020D8F00020D8F0071
:100D0B00020D8F00020D8F00020D8F00020D8F0060
:100D1B00020D8F00020D8F00020D8F00020D8F0050
:100D2B00020D8F00020D8F00020D8F00020D8F0040
:100D3B00020D8F00020D8F00020D8F00020D8F0030
:100D4B00020D8F00020D8F00020D8F00020D8F0020
:100D5B00020D8F00020D8F00020D8F00020D8F0010
:100D6B00020D8F00020D8F00020D8F00020D8F0000
:100D7B00020D8F00020D8F00020D8F00020D8F00F0
:100D8B00020D8F0074551216F8C22322901401E045
:100D9B00B4FE03020DBBB4FF03020DE9B400030262
:100DAB000DE9B4FD03020DE974551216F8C22322A6
:100DBB00120DC674AA1216F8C223227A07900000ED
:100DCB007400F0A3DAFCD226D225751800751E1418
:100DDB00751F007400900005F07408A3F022C21E6A
:100DEB00F5F0202606900000E07003020EB4FBF530
:100DFB001F7A01A9F0EA75F008A4240FF582E5F03B
:100E0B003400F58389F0E0B5F0028003020EA7D21F
:100E1B001EE582C39403F582E5839400F583E0FC21
:100E2B00A3E0FDA3E0F9E51FC39A04C0F075F00839
:100E3B00A4AFF0FEEA1475F008A42410F8E5F03422
:100E4B0000F5A0EA75F008A42410F582E5F0340053
:100E5B00F583120EEBECF8EDF5A0E92CF58274009E
:100E6B003DF5837400C39582FE74149583FF120EB7
:100E7B00EB900003E0C399F0A3E09400F0A3E0C370
:100E8B0099F0A3E09400F0120EFAD0F01B151FE5B9
:100E9B001FB40003020DBBBB000C800D0ABB00028C
:100EAB008007DB028003020DFE301E06E51F90005B
:100EBB0000F074AA1216F8C22322A85C9000617984
:100ECB0000E993601175A01FF20908E8B55BF220E9
:100EDB0020FAD29980F6885C202002D299C2232274
:100EEB00E0F2121E7EDEF9BF00028002DFF22290DA
:100EFB000014E51F6029F8E0C39CAE82AF83A3E02A
:100F0B009505400D8E828F83E0C399F0A3E094008A
:100F1B00F074072582F58274003583F583D8D822C7
:100F2B00900000E0F5F0FA7B007E0D900003E02AC4
:100F3B00FA74003BFBA3DEF6900010AEF0BE00038C
:100F4B00020F5C7F08E02AFA74003BFBA3DFF6DE9E
:100F5B00F2900003E0FFA3E0FE900800EE4F600F5D
:100F6B00E02AFA74003BFBA31FBFFFF01E80ED7E4F
:100F7B000F901500E02AFA74003BFBA3DEF67E0F00
:100F8B0090150FE02AFA74003BFBA3DEF67E20904F
:100F9B001546E02AFA74003BFBA3DEF6900001EA4B
:100FAB00F0A3EBF022900000E004B4FE087455129D
:100FBB0016F802104EF014F5F07408A42410F8E59E
:100FCB00F03400F5A07A04901401E0F2121E7EDAE0
:100FDB00F9E0B4FE0E900000E014F074551216F810
:100FEB0002104EFDA3E0FCA3A982AA83900003E0AC
:100FFB002CF0A3E03400F0900005E0F5F0F2121EA7
:10100B007EE0F2FB121E7EECF2121E7EEDF2121E41
:10101B007E74FFF2121E7EF2121E7EF2121E7EF202
:10102B008A838982A9F0E08BA0F3A309B900010B95
:10103B00DCF4900005E9F0A3EBF0C226C22574AAFC
:10104B001216F8C22322202606202503120BA874A1
:10105B00AA1216F8C22322121DF374AA1216F8C292
:10106B002320340B901522E04402F090E000F0D2E4
:10107B0097D29622121C221221A612160F74AA12B4
:10108B0016F8C22322901401E0B4400040028013F2
:10109B00B40A00400E900007F0121DF374AA12164A
:1010AB00F8800574551216F8C22322901401E0B48F
:1010BB000A0040028022FA780075A015F2121E7EFB
:1010CB00E0B43F005012B43200400DF2DAEF74AAD4
:1010DB001216F8121DF3800A901500E4F0745512E5
:1010EB0016F8C22322780175A0149015467D20E2D4
:1010FB00F0121E7EDDF9121DF31221A612160F74CB
:10110B00AA1216F8C2232290155CE0547FF56B905F
:10111B001401E05407F569901402E0B41B0040027F
:10112B00741AF56AC22322900009E075F01E700351
:10113B0075F018B4010375F019901401E0B41800A0
:10114B004001E4901585F0901402E0B43C0040019E
:10115B00E4901586F0901403E0B43C004001E49059
:10116B001587F0901404E0B5F0004001E490158869
:10117B00F0D23DC22322901401E0700575F0188067
:10118B0060B4010575F0198058B4020575F01E8026
:10119B0050B4030575F01E8048B4040575F01E802D
:1011AB00407402900009F090150F7400F0A37400C6
:1011BB00F0A37400F0A37400F0A37418F0A37400F0
:1011CB00F0A37400F0A37400F0A37400F0A37400F8
:1011DB00F0A37400F0A37400F074551216F8021209
:1011EB00DD900009F0901402E0B4180050B3901594
:1011FB000FF0F555901517F0901403E0B43C005028
:10120B00A0901510F0F556901518F0901404E0B45A
:10121B003C00508D901511F0F557901519F0901466
:10122B0005E0B5F00040030211AC901512F0F55833
:10123B0090151AF0C223901406E0B41804D2238040
:10124B000540030211AC901513F0F530901407E034
:10125B00B43C0040030211AC30230560030211AC17
:10126B00901514F0F531901408E0B43C00400302E3
:10127B0011AC30230560030211AC901515F0F5325B
:10128B00901409E0B5F00040030211AC3023056067
:10129B00030211AC901516F0F53390140AE0A2E09E
:1012AB009222A2E19205A2E2921FA2E3922AA2E469
:1012BB00922BA2E5922DA2E6922EA2E7921390001A
:1012CB0008F0D296202204C2018002D20174AA1225
:1012DB0016F8121DF31221A612160F122153C22358
:1012EB0022900009E075F01E700375F018B401032D
:1012FB0075F019901401E0B4180040028047901467
:10130B0002E0B43C004002803C901403E0B43C008B
:10131B0040028031901404E0B5F00040028026902A
:10132B00151AF0901403E0901519F0901402E09048
:10133B001518F0901401E0901517F074AA1216F816
:10134B00121DF3800574551216F8C2232290140156
:10135B00E0FA743F2AFA7902122083C223229014F6
:10136B0001E0FBA3E0FA901522E04AF0FAA3E04B70
:10137B00F090E800F090E000EAF074AA1216F8C2C0
:10138B002322901401E0F4FBA3E0F4FA901522E081
:10139B005AF0FAA3E05BF090E800F090E000EAF07E
:1013AB0074AA1216F8C2232290E800E0FB90E0002A
:1013BB00E0FA74AA1216F8EB1216F8EA1216F8C233
:1013CB002322D201D29174AA1216F8C2232220151D
:1013DB001720001DC23F302218301F15301C04D2BD
:1013EB0001801D121B558009103F028004D2018021
:1013FB000FD291C201C200C21574AA1216F8C223F1
:10140B0022202B04D200C29174AA1216F8C22322F6
:10141B00302206C2AFD215D2AF74AA1216F8C2236D
:10142B0022901401E0A2E0921D900008E092E3C22A
:10143B001D5002D21DF075A015781B901402E0F917
:10144B00F208A3E0FAF208A3E0F2FBC3740099746C
:10145B008D9A74279B4003021480C21D900008E0F4
:10146B0054F7F090151B7400F0A3F0A3F074551211
:10147B0016F8021488121DF374AA1216F8C223224E
:10148B00900000E0FFFA1216F89000100FDF0280B8
:10149B004EE01216F82AFAA3E01216F82AFAA3E085
:1014AB001216F82AFAA3E01216F82AFAA3E0FDA303
:1014BB00E0FEA3E0FCA3E0A31216F82AFAEC121646
:1014CB00F82AFAC082C0838D828E830CDC028009DD
:1014DB00E01216F82AFAA380F3D083D08280AEEA0A
:1014EB001216F8C223227F037E007A00903400E0AC
:1014FB001216F82AFAA3DEF7DFF59020007E10E033
:10150B001216F82AFAA3DEF7EA1216F8C223229073
:10151B0015657F20E4F0A3DFFC756700C234C2358C
:10152B00C236901522E04402F090E000F074AA124B
:10153B0016F8C22322E4303502440130360244024D
:10154B00FA1216F89015657F20E01216F82AFAA306
:10155B00DFF7EA1216F8C22322901401E0541F752C
:10156B00F010A42400F582E5F03435F58375A01452
:10157B007801121C0DA85E12214CB4100040F8909B
:10158B0014011215C074AA1216F8C223227C20EC87
:10159B001475F010A42400F582E5F03435F583E0E2
:1015AB0030E70FA85E12214CB41000500280F612E7
:1015BB0015C0DCDB22E0D2E775A018F2FB75A01793
:1015CB007401F20875A0187400F275A017F208A345
:1015DB007A0DE075A018F22BFB75A0177400F208BA
:1015EB00A3DAEF75A018EBC313F275A0177400F212
:1015FB0008885E75A080790274B5F375A0807905B3
:10160B007406F32212214CB4080040F874BF855EB7
:10161B0082758318F0FB7583177401F074030582D0
:10162B00758318F02BFB758317E4F0E430680274B4
:10163B00010582758318F02BFB758317E4F0E52BFE
:10164B000582758318F02BFB758317E4F0C082902D
:10165B000009E0D0820582758318F02BFB75831788
:10166B00E4F0E5350582758318F02BFB758317E4E1
:10167B00F0E5340582758318F02BFB758317E4F0C6
:10168B000582758318EBC313F0758317E4F005829D
:10169B0085825E90800274B5F09080057406F0220E
:1016AB00FBE55EC3955DF4B4030050030216ACEB8F
:1016BB00A85E75A018F275A0177401F20875A01832
:1016CB00E5F0F22BFB75A0177400F20875A018EB70
:1016DB00C313F275A0177400F208885E75A08079A9
:1016EB000274B5F375A08079057406F322C0E0C0CF
:1016FB0082C08375831F855C82F0E55C04F583B53E
:10170B005B072020FAD29980F685835C202002D2D9
:10171B0099D083D082D0E02275A891C28CC28EC2A0
:10172B008F902E7B12026D902E8B12026D902EB32A
:10173B0012026DC20BC20DC212C20FC20CC210C27A
:10174B000EC207851211758A00754C0075294075FC
:10175B002A0175550075560075570075580075337D
:10176B000090151BE0F530A3E0F531A3E0F532C294
:10177B00AF75B80675A81FD246D28CD2AFC2231252
:10178B00054730230D75A891C28CC28E120C7D02B9
:10179B00195D100C183004E7C20412030A1207A2D9
:1017AB003001DC75A891C28CC28E02195DE53954EB
:1017BB000375F00AA4F8E538540F28200E09B41568
:1017CB00BED20E7A0080B8F89017DBEA540323736D
:1017DB008006800A800E8028B816660A80A1B8178A
:1017EB00600A809BB818030A8095B8005475461898
:1017FB0075120075295BC206902EF612026D80469B
:10180B00B8192875461E751200752915C206902F3A
:10181B000812026DE53930E20AD206902F1112023E
:10182B006D8023902F1A12026D801BB80013754622
:10183B001975120075294DC206902EFF12026D808C
:10184B0005C20E02178A902E9912026DC2AF854304
:10185B0041854442D2AFE54175F014A4F541A8F09F
:10186B00E54275F014A428F542754E00754D00D273
:10187B0010D20FE539540375F00AA4F5F0E538548E
:10188B000F25F004F548F554E53B540775F00AA411
:10189B00F5F0E53A540F25F0F549F553E53D5407BE
:1018AB0075F00AA4F5F0E53C540F25F0F54AF55216
:1018BB00E53F540375F00AA4F5F0E53E540F25F00F
:1018CB00F54BF551D23AC202C218C2191205473074
:1018DB00230302179020100C75A891C28CC28E7531
:1018EB002800806E301902C219301836C218120740
:1018FB00A230010975A891C28CC28E8055300D0B98
:10190B00120A82902E9912026D8017902EA6120247
:10191B006DD296E511600BD51108D236C201C222E9
:10192B00803030021DC202301603120ACB301B036B
:10193B00120B3E1208B23013031222A012030A122A
:10194B00029130170AC217301605C216120AFC0292
:10195B0018D7D296901522E04409F090E000F002DF
:10196B000192C21575A891901522E054FEF090E0FB
:10197B0000F0902E8312026DC28CC28EC23FC21A2F
:10198B00C218121B5520426420413A20402575464F
:10199B0018754000901554E0B4E90C902EF6120225
:1019AB006D901554021A0A902EED12026D9015547B
:1019BB00021A0A902EFF12026D9015567546197574
:1019CB004000021A0A304012902F0812026D901537
:1019DB005A75461E754000021A0A902F1112026D9D
:1019EB0090155875461E754004021A0A902F1A124C
:1019FB00026D90155875461E754000C240C241E0FD
:101A0B00A3750F00F50EE0F50D8000754700750905
:101A1B0036750C00750B0A750A01D209850E4FC27B
:101A2B00AF75B802E4C3954FF58A202E0D902EC6E4
:101A3B0012026D75A81BD28C805775A81FC28B9094
:101A4B002E8B12026D902EE012026D20412F204042
:101A5B0016902EED12026D74EA750F00F50E850EC1
:101A6B004F74C2F50D802A902EFF12026D750F0078
:101A7B0074E0F50E850E4F7497F50D801474BA75DE
:101A8B000F00F50E850E4F74F0F50D902F1A120204
:101A9B006DC246C28DC28FD2AFC223D21C12054774
:101AAB00302306120C7D20012E300211C2021208C7
:101ABB00B23013031222A012030A1202913018DD66
:101ACB00C2181207A220010F30150AC292902ED312
:101ADB0012026D800E80C675A891C28CC28E7528BD
:101AEB00008055120547202314300226C202120330
:101AFB000A1207A2301506200132201515D29220AA
:101B0B002E08902EC612026D8093902EE012026D5D
:101B1B00808B3018CEC21880CAD29175A891C28C16
:101B2B00C28ED201752800120C7D800CD29175A843
:101B3B0091C28CC28E752800901522E04401F09062
:101B4B00E000F0D296C21C02019290150FE0F55501
:101B5B00A3E0F556A3E0F557A3E0F558A3E0F53065
:101B6B00A3E0F531A3E0F532A3E0F533A330000396
:101B7B0090150FE0F54BA3E0F54AA3E0F549A3E080
:101B8B00F548303D12901585E0F54BA3E0F54AA3DF
:101B9B00E0F549A3E0F548900009E0B4000875288A
:101BAB00007568048027B4010875280175680480E6
:101BBB001CB403087528047568018011B4040875FA
:101BCB00280275680180067528037568017536FC57
:101BDB007537BFE54875F00A8485F0384540F5390F
:101BEB00E54975F00A8485F03AF53BE54A75F00A4C
:101BFB008485F03CF53DE54B75F00A8485F03EF5A8
:101C0B003F227A108003121E7EE2F0DAF9FAE0C36B
:101C1B009A70FB121E7E22120DC6121DAA90344022
:101C2B00E0B4550D902000E0FCB4FE004006021C11
:101C3B00CF021D22902003E0A3F8C3740098E0F8B4
:101C4B00740C985003021CCF90200075A0007800F4
:101C5B00ECF27D00FE121E7EE0FBF2121E7EE0FA1D
:101C6B00F2121E7E7F0DE0F22CFC74003DFD121E65
:101C7B007EDFF3BE0004D226804AC2269020107865
:101C8B001075A0007F08E0F22CFC74003DFD121EC5
:101C9B007EDFF3DEEF7E08E0F2121E7EDEF99000AF
:101CAB0003E0FFA3E0FE90280075A0087800EE4F3C
:101CBB006012E0F2121E7E2CFC74003DFD1FBFFF74
:101CCB00ED1E80EA7F0F780075A015903400E0F2CE
:101CDB00121E7E2CFC74003DFDDFF37F0F780F7519
:101CEB00A015903410E0F2121E7E2CFC74003DFD0A
:101CFB00DFF37F20784675A015903420E0F2121E9A
:101D0B007E2CFC74003DFDDFF3ED8AF0B5F008ECA2
:101D1B008BF0B5F0028030901522E054FDF090E08E
:101D2B0000F0D235C297C296122DD9122DD9D29767
:101D3B00D2967C209034FF7A107400A3F0DAFCE08A
:101D4B00B400FCDCF28010900000E06006C226D2EA
:101D5B00258004D226C2257D04785590150FE0F618
:101D6B00A308DDFA7D047830901513E0F6A308DDA7
:101D7B00FA900008E0A2E09222A2E19205A2E29280
:101D8B001FA2E3922AA2E4922BA2E5922DA2E69245
:101D9B002EA2E79213202204C2018002D2012290CC
:101DAB002E0275A00078007A10E493F2121E7EDAF0
:101DBB00F8902E1275A01578007A0FE493F2121E8C
:101DCB007EDAF8902E3375A015780F7A0FE493F224
:101DDB00121E7EDAF8902E1D75A01578467A16E441
:101DEB0093F2121E7EDAF822202606202503120B10
:101DFB00A8120F2B780075A000902000E2FC121C9B
:101E0B000DEC7003021E47C31304FC121C0DDCFB0C
:101E1B00900003E0FCFFA3E0FD7A04EDC313FDEC9F
:101E2B0013FCDAF7EF540F60010CBC0002800D7845
:101E3B000075A008902800121C0DDCFB780075A023
:101E4B0015903400121C0D780F75A01590341012DC
:101E5B001C0D784675A015903420121C0D78567504
:101E6B00A015903430121C0D9034407455F0E0B432
:101E7B0055FC22A308B8000205A022901537E054A8
:101E8B000F2323901E9273021ED300021EED00023D
:101E9B001FD90002202E000220530002205F0002F7
:101EAB00206B00022077000220E2000220FC0002DF
:101EBB0021160002213100021ED200021ED20002A6
:101ECB001ED200021ED20022901537E05430FA3396
:101EDB004A5450FAA3E0543F901524F0901525EA8C
:101EEB00F022901538E0543FD2E7FA901524E0F930
:101EFB00901525E0F5F0301D048A58893312214CDA
:101F0B00B4050040F8758318855E82EAF075831777
:101F1B007401F005827583187401F02AFA75831722
:101F2B007400F00582758318E5F064400354204576
:101F3B00F0202207200D09440880053001024408D7
:101F4B00F02AFA7583177400F00582758318E9542B
:101F5B003FF02AFA7583177400F00582758318EA2F
:101F6B0003547FF07583177401F0058285825E90B0
:101F7B00800274B5F09080057406F0C22122122104
:101F8B004CB40300500280F6758318855E82EAF02C
:101F9B007583177401F005827583187408F02AFA9B
:101FAB007583177400F00582758318EA03547FF06C
:101FBB007583177401F0058285825E90800274B57B
:101FCB00F09080057406F0C22122743F8006C22176
:101FDB00901538E0543FD2E7FA12214CB40300506D
:101FEB000280F6758318855E82EAF075831774019B
:101FFB00F005827583187408F02AFA75831774003C
:10200B00F00582758318EA03547FF075831774010A
:10201B00F0058285825E90800274B5F09080057425
:10202B0006F022901538E0543FFA901526E0B40ADA
:10203B0002801204F0F9E58229F58274003583F5EC
:10204B0083EAF0D21BC22122901538E0543FFA7973
:10205B0018022083901538E0543FFA791902208337
:10206B00901538E0543FFA791A022083901538E026
:10207B00543FFA791B022083E562C39561F4B405E2
:10208B0000500280F375831C75A01B85628274FF60
:10209B004480FBF07401A882F205827400F02BFBE4
:1020AB007400A882F20582E9547FF02BFB7400A820
:1020BB0082F20582EAF02BFB7400A882F20582EB18
:1020CB0003547FF07401A882F205828582629060CE
:1020DB00057406F0C22122901537E0232354C0F972
:1020EB00A3E0543F49F9901522E049F090E000F04D
:1020FB0022901537E0232354C0F9A3E0543F49F94C
:10210B00901523E049F090E800F022901537E0237A
:10211B002354C0F9A3E0543F49F4F9901522E05938
:10212B00F090E000F022901537E0232354C0F9A380
:10213B00E0543F49F4F9901523E059F090E800F092
:10214B0022E55EC3955DF4229060027415F09060F9
:10215B0000202D04741B80027413F07407F0A3206D
:10216B002D0474BB800274CCF09060047408F09062
:10217B0060027405F09060057406F090800274158F
:10218B00F0908000741BF07407F0A374CCF0908077
:10219B00047408F09080057404F022901546E0A2B8
:1021AB00E09203A3A3A3A3A3E0FA5407239021BCBB
:1021BB007321CC21DD21EE21FF4110412141324120
:1021CB00327403904000F07400904003F0752B00C4
:1021DB0080667404904000F07401904003F0752BFE
:1021EB000080557405904000F07401904003F07529
:1021FB002B0080447406904000F07401904003F073
:10220B00752B0080337404904000F07401904003F0
:10221B00F0752B0180227405904000F07401904002
:10222B0003F0752B0180117406904000F07401903F
:10223B004003F0752B018000EA5470C42390224CAC
:10224B0073416C416C416C416C415C4164416C412C
:10225B006C7404904001F0800E7405904001F08086
:10226B00067406904001F0EAA2E7929592689000FE
:10227B0009E0B4000590154C8013B4010590154E80
:10228B00800BB402059015528003901550E0F53584
:10229B00A3E0F53422C0D0C0E0C0F0C082C083E51B
:1022AB005EC3955DF4B40700500302233F7583189A
:1022BB00855E8274BFF0F5F07583177401F00582AB
:1022CB00758318740DF025F0F5F0758317E4F005A0
:1022DB0082758318E54BF025F0F5F0758317E4F064
:1022EB000582758318E54AF025F0F5F0758317E440
:1022FB00F00582758318E549F025F0F5F075831725
:10230B00E4F00582758318E548F025F0F5F0758348
:10231B0017E4F00582758318E5F003547FF075839D
:10232B0017E4F0058285825E90800274B5F0908090
:10233B00057406F0D083D082D0F0D0E0D0D022202C
:10234B004608B227302702D28C32C0D0C0E0D2145C
:10235B00300D02B2967402C28CC58AD28CF54FE452
:10236B00C54C308D070470027403C28DF550C3E564
:10237B004F948AE5509400401BC3E529954FE52AFD
:10238B0095504004D208801374B5954F7402955044
:10239B00C2085007C20BC20D02247030080D300763
:1023AB000A200A28C2070547022470200B71A208D5
:1023BB00E53713F537E53613F536B4FC7EE537B460
:1023CB00BF79300807D20AD20702247020B5FD303E
:1023DB00B5FDC294D2177400B54808B54905B54A86
:1023EB00028016E53F540775F00AA4F5F0E53E545C
:1023FB000F25F0F54BF551D23A750938750B087569
:10240B000A08754700D20BC20AC207300F57754531
:10241B0000754E00754D00D28ED28FC20F8046C014
:10242B0000A208A809E613F6D000D50A0E05097517
:10243B000A08D50B06C20BD20DD20C300804D207FA
:10244B0080230547C207E54354F02544C4F50FE547
:10245B004F54F02550C4254350020544C3950FF546
:10246B004350021544D0E0D0D03220460302248BD7
:10247B00C0E0054CE54C7005D204754C03D0E0323E
:10248B00C0D0C0E0C0F0C082C08330091130150746
:10249B00300504D2968002B296C20702253CC000DA
:1024AB00A809E630E00E301507300504D2968002FD
:1024BB00B296D20703F6D0000547E50AC333F50AF7
:1024CB00506F750A010509D50B67750936750B0A2F
:1024DB00754700854854854953854A52854B51D2DF
:1024EB003AE54875F00A8485F0384540F539E549F9
:1024FB0075F00A8485F03AF53BE54A75F00A848558
:10250B00F03CF53DE54B75F00A8485F03EF53FD286
:10251B008F302E1DD5681AB209050CC28C758AFE38
:10252B00756801E5285407B40200502F75680480C4
:10253B002AB209850E4FE50CC3950D4002054F05D8
:10254B000CC28CE4C3954F258AF58AD28C201A0BCA
:10255B00E509B43B06D21AD218D294D083D082D0DC
:10256B00F0D0E0D0D0322046030227D6C0D0C0E056
:10257B00E54E6004154E8019E54D601AC3E4954D88
:10258B00754D00C28E258C5004D28E8009F58CD2ED
:10259B008ED0E0D0D032C21AE545700D200D13203D
:1025AB00B5FD30B5FDC2948009B40206D21AD2949F
:1025BB00D218C0F0C083C082200D030226FE201A61
:1025CB000C101406C20DC20BD20F0226FE53A8FB31
:1025DB00854C17858A16E547A20785441485431554
:1025EB0043A8049211F5F0B42800400302267CC3E3
:1025FB00742895F023F5139415400BC20DC212C22B
:10260B000BD20F0226FEE514C313C51513F51420C8
:10261B00110BC39516E5159517400280021513E5AE
:10262B00148513F0A4F51685F017E5158513F0A4A2
:10263B002517C313C51613C516C313F517E51613C4
:10264B00F516E517C313F515E51613C515C313C515
:10265B001513F5142541F541E5153542F542E516FF
:10266B002541F54DE5173542F54E154ED212022791
:10267B0006942823F5139415400BC20DC212C20BFE
:10268B00D20F0226FEE514C313C51513F514201142
:10269B000BC39516E5159517400280020513E5143B
:1026AB008513F0A4F51685F017E5158513F0A42511
:1026BB0017C313C51613C516C313F517E51613F574
:1026CB0016E517C313F515E51613C515C313C51575
:1026DB0013F514C3E5419514F541E5429515F54203
:1026EB00C3E5419516F54DE5429517F54E154ED2BE
:1026FB0012800885424E85414D154EE545B40302C7
:10270B008008B40102D2190227C6300D5830125579
:10271B00901522E054F6F090E000F0851211E539A7
:10272B00540375F00AA4F5F0E538540F25F0F5487D
:10273B00E53B540775F00AA4F5F0E53A540F25F084
:10274B00F549E53D540775F00AA4F5F0E53C540F47
:10275B0025F0F54A7400B54817B54914B54A11056B
:10276B0048054B8046901522E04408F090E000F0BD
:10277B000548E548B546347548000549E549B43C7C
:10278B002A754900054A300610E54A75F00A84E5BA
:10279B00F0600674022548F548E54AB43C0D754ACD
:1027AB0000054BE54BB41803754B00854854854920
:1027BB0053854A52854B51D202D23A0545534503B4
:1027CB00D082D083D0F0D0E0D0D032C0D0C0E0C027
:1027DB00F0C083C082301503022874203D3D0548AC
:1027EB00E548B5464A7548000549E549B43C40758E
:1027FB004900054A30411020400DE54A75F00A8426
:10280B00C5F06003754802E54AB43C23754A0005E0
:10281B004BE54BB41819754B008014901585E0F5FA
:10282B004BA3E0F54AA3E0F549A3E0F548C23DE52B
:10283B004BB53035E54AB53130E549B5322BE54876
:10284B00B53326D291302B0D200506D215D23F8001
:10285B0018D20180143000052005F680EE85554B0B
:10286B0085564A855749855848D202C21A20B5FD6C
:10287B0030B5FDC294D082D083D0F0D0E0D0D0322E
:10288B00E564C3956385631BB407005003022C6B8F
:10289B00122C6CB4F075122C6C20E76DB47F6C129B
:1028AB002C6C20E764B47F02800B2409F5F09000B8
:1028BB0007E0B5F056122C6C20E74EB4024D122CEB
:1028CB006C20E745B410028008B430028003B47F5B
:1028DB003A122C6C20E732F51AB401030229DAB450
:1028EB0002030229DAB403030229DAB41503022A1C
:1028FB0056B41603022A56B41703022A56B4180309
:10290B00022A56B41905022919151B022C65E56418
:10291B00C39563B412005003022C6B122C6C20E78E
:10292B00E8C3943075F00AA4F5F0122C6C20E7D9AB
:10293B00C3943025F0B418004001E4901585F012D3
:10294B002C6C20E7C4B400C3122C6C20E7BBC394DF
:10295B003075F00AA4F5F0122C6C20E7ACC3943060
:10296B0025F0B43C004001E4901586F0122C6C204D
:10297B00E797B40096122C6C20E78EC3943075F059
:10298B000AA4F5F0122C6C20E73FC3943025F0B469
:10299B003C004001E4901587F0122C6C20E72AB420
:1029AB00002A122C6C20E721C3943075F00AA4F591
:1029BB00F0122C6C20E712C3943025F0B41F0040AA
:1029CB0001E4901588F0022A56022914022916E513
:1029DB0064C39563B40F005003022C6B122C6C2054
:1029EB00E7E7C3943075F00AA4F51C122C6C20E7B2
:1029FB00D8C39430251CF51C122C6C20E7CBB400EB
:102A0B00CB122C6C20E7C2C39430F51D122C6C201A
:102A1B00E7B7B400B7122C6C20E7AEC3943075F057
:102A2B000AA4F51E122C6C20E79FC39430251E754B
:102A3B00F00AA4F51E85F01F122C6C20E78BC394B3
:102A4B0030251EF51EE51F3400F51F122C6C30E7E8
:102A5B0044B4F744E51AB40104C201806AB403021A
:102A6B008065B40203022B8AB41530D291C20120C7
:102A7B001510200019C23F302214301F11121B55A4
:102A8B00800C103F028007C2AF121B55D2AFC200A1
:102A9B00C215022BDB022C65022914B4160C302252
:102AAB00EDC2AFD215D2AF022BDBB41705D20102A8
:102ABB002BDBB4180A202B04D200C291022BDBB4FF
:102ACB001902D23D022BDB12214CB40500500280BF
:102ADB00F6758318855E82E51C4480F519B4810078
:102AEB004000F07583177401F00582758318E51D9E
:102AFB00C3C23E9403400EF51D94034004F51DD252
:102B0B003E740D80027401F02519F5197583177445
:102B1B0000F00582758318E51E33E51F3330E202A2
:102B2B0044105413C51D600920E1047440800274E5
:102B3B0020451DF51DE51AB403067408451DF51D4A
:102B4B00E51D103E024408F02519F519758317741D
:102B5B0000F00582758318E51E547FF02519F519D1
:102B6B007583177400F00582758318E51903547F7C
:102B7B00F07583177401F0058285825E022BCF12EC
:102B8B00214CB40300500280F6758318855E82E5F4
:102B9B001C4480F519F07583177401F00582758359
:102BAB00187408F02519F5197583177400F0058250
:102BBB00758318E51903547FF07583177401F005BD
:102BCB008285825E90800274B5F09080057406F069
:102BDB0074F075831C856282F0740075831BF0059D
:102BEB0082E56165826073858262747F75831C8563
:102BFB006282F0740075831BF00582E5616582606B
:102C0B0059858262740375831C856282F07400752A
:102C1B00831BF00582E5616582603F8582627402E9
:102C2B0075831C856282F0740075831BF00582E549
:102C3B00616582602585826274F775831C8562826B
:102C4B00F0740075831BF00582E5616582600B856E
:102C5B0082629060057406F08000851B6302288BEE
:102C6B002275831A851B82E0051B22C0D0C0E0C0F1
:102C7B0082C08310990C109829D083D082D0E0D0D9
:102C8B00D032C299E55B655C7005C220022CAAD2DA
:102C9B0020855B82055B75831FE0F5997598D002E3
:102CAB002C7EE59975831E855A82F075831D209ABB
:102CBB0004740080027401F0A3E5596582600385FA
:102CCB00825A022C7EC0D0C0E0C082C083908005A7
:102CDB00E030E103022D76908005E030E203022D17
:102CEB00C1906005E030E103022D0B906005E030F0
:102CFB00E205022D4A80D6D083D082D0E0D0D032EC
:102D0B00E561656270099060057404F0022CF62091
:102D1B002D1D9060027415F075831B856182E06038
:102D2B0008906000741FF08006906000741BF075B3
:102D3B00831C856182E0906003F00561022CF690A4
:102D4B006001E075831985648220E50474008002BC
:102D5B007401F0906003E075831A856482F0A3E53B
:102D6B006365826003858264022D00E55D655E709C
:102D7B000F9080057404F090800274A5F0022CE291
:102D8B009080027415F0758317855D82E060089062
:102D9B008000741FF08006908000741BF075831800
:102DAB00855D82E0908003F0055DB48100400400F6
:102DBB00000000022CE2908003E075831685608290
:102DCB00F0A3E55F65826003858260022CEC7A3E9E
:102DDB00EAC0E0122DE7D0E0FADAF5227A007B2088
:102DEB00DAFEDBFC227A007B0ADAFEDBFC227A00BD
:102DFB007B32DAFEDBFC22000000000000080A0236
:102E0B0002000000000000000000000000000000B5
:102E1B00000000000100040047C744E8397B396C0F
:102E2B00EE00E5CDBECEBD00000000001800000096
:102E3B0000000000008D2701014469676974616C13
:102E4B002042696E6C6F6F7020000201496E6974CD
:102E5B0069616C697A696E672E2E2E20000201560D
:102E6B00657273696F6E20352E3030202020200064
:102E7B000101526561642000010147656E2020004D
:102E8B0001062D2D3A2D2D3A2D2D2E2D2D00020123
:102E9B004C6F636B65642020202000020153656C2E
:102EAB00662047656E2020000201417761697469D5
:102EBB006E6720534D505445202000020152756E11
:102ECB006E696E6720202000020149646C696E6791
:102EDB0020202020000201562D53796E63202020E4
:102EEB002000020B32332E39373600020B323420DE
:102EFB0066707300020B32352066707300020B3361
:102F0B00302066707300020B32392E3937640002A1
:082F1B000B32392E39376E002C
:00000001FF
